:0A0000007A2C000000000000002828
:10000A008312D903D9035908003C03181128D903CC
:10001A0000000000000008280000000000000000A6
:04002A0000000800CA
:10002E00FB09FA09F909F809F80A0319F90A03197B
:08003E00FA0A0319FB0A08008D
:100046007408F8027508031C750FF9027608031C7C
:10005600760FFA027708031C770FFB02F30D0730C1
:10006600FC00730DF80DF90DFA0DFB0D7408731CE9
:100076004A28F8027508031C750FF9027608031C56
:10008600760FFA027708031C770FFB025728F8074A
:1000960075080318750FF90776080318760FFA071F
:1000A60077080318770FFB07F30DFC0B3428720D46
:1000B600F80DF90DFA0DFB0D7408731C7028F80283
:1000C6007508031C750FF9027608031C760FFA02F1
:1000D6007708031C770FFB027D28F80775080318BD
:1000E600750FF90776080318760FFA0777080318CD
:1000F600770FFB07F20D0730FC00720DF80DF90DB6
:10010600FA0DFB0D7408721C9628F8027508031C7C
:10011600750FF9027608031C760FFA027708031C9E
:10012600770FFB02A328F80775080318750FF90760
:1001360076080318760FFA0777080318770FFB0778
:10014600F20DFC0B8028710DF80DF90DFA0DFB0D63
:100156007408721CBC28F8027508031C750FF90296
:100166007608031C760FFA027708031C770FFB024A
:10017600C928F80775080318750FF90776080318D4
:10018600760FFA0777080318770FFB07F10D07308C
:10019600FC00710DF80DF90DFA0DFB0D7408711CBC
:1001A600E228F8027508031C750FF9027608031C8D
:1001B600760FFA027708031C770FFB02EF28F80781
:1001C60075080318750FF90776080318760FFA07EE
:1001D60077080318770FFB07F10DFC0BCC28700D81
:1001E600F80DF90DFA0DFB0D7408711C0829F802BB
:1001F6007508031C750FF9027608031C760FFA02C0
:100206007708031C770FFB021529F80775080318F2
:10021600750FF90776080318760FFA07770803189B
:10022600770FFB07F00D0730FC00700DF80DF90D88
:10023600FA0DFB0D7408701C2E29F8027508031CB4
:10024600750FF9027608031C760FFA027708031C6D
:10025600770FFB023B29F80775080318750FF90796
:1002660076080318760FFA0777080318770FFB0747
:10027600F00DFC0B182970184E297408F80775083C
:100286000318750FF90776080318760FFA0777082B
:080296000318770FFB070800B5
:0C029E00831238088A003708820008002C
:1002AA0083125708F2007208F000F20A70088400FC
:1002BA00000803196129582957087202F000013011
:0A02CA00F002F101031CF10308002B
:1002D4008312570883169B009C131C141A08F00001
:0202E400080010
:0C02E6000E30FD00FD0B75290000080023
:1002F20083120313F801F9011030FC00710DF80D9F
:10030200F90D7408F8027508031C750FF902031839
:1003120091297408F80775080318750FF907031077
:0A032200F00DF10DFC0B7F2908001F
:10032C00831203132230FC00F801F901FA01FB01DE
:10033C00FC030319CC290310FB0CFA0CF90CF80C78
:10034C00F30CF20CF10CF00C031C9E29FC030319AA
:10035C00BE297408F80775080318750FF907760895
:10036C000318760FFA0777080318770FFB07A229F3
:10037C007408F80775080318750FF9077608031841
:0E038C00760FFA0777080318770FFB070800B3
:10039A0040308312F0001F30F100F201F30108002F
:1003AA0001308312D8003608D7064308840036087D
:1003BA00003A0319E3293F088004E529400880052B
:1003CA003308D9000520D70958080319012A580803
:1003DA005705F000031DF4293F088004F629400858
:1003EA008005D80D581002303302D90005200000CC
:1003FA00000000000000E9293608003A0319082A1B
:10040A00400880050A2A3F0880043308D9000520DD
:02041A000800D8
:10041C0083120313FC01F71BFC0AFD01FB01FA011B
:10042C00F901F80173087204710470040319A22A0B
:10043C0073087706C400C41BFD09F71F302AF409A2
:10044C00F509F609F709F40A0319F50A0319F60A6E
:10045C000319F70AF31F3D2AF009F109F209F30910
:10046C00F00A0319F10A0319F20A0319F30A7308C3
:10047C007704C400C41B5E2A2320FC1B7B2AFD1FAF
:10048C00A22AF009F109F209F309F00A0319F10A99
:10049C000319F20A0319F30AF809F909FA09FB0915
:1004AC00F80A0319F90A0319FA0A0319FB0AA22A12
:1004BC00F71F752AF31B6F2A7308FB007208FA00EA
:1004CC007108F9007008F800F301F201F101F00174
:1004DC00452AF301F201F101F001F00A0034F309AD
:1004EC00F209F109F009FC17422AF80A0319F90A72
:1004FC000319FA0A0319FB0A74087802031D452A2A
:10050C0075087902031D452A76087A02031D452ACF
:10051C0077087B02031D452AFB01FA01F901F8015A
:10052C00F00A0319F10A0319F20A0319F30AF31F6B
:10053C00452AC4014416FF34C4017C1CA62A17208A
:04054C00003E080065
:100550008312C801053048020318B52A4808470726
:10056000840020308000C80AAA2A4808470784006F
:100570008001C80348084707C9000A30F400F501A4
:100580004508F0004608F10079217808F000790864
:10059000F1003030F00749088400700880000A300C
:1005A000F400F5014508F0004608F10079217008D3
:1005B000C5007108C60000307106031DE12A003035
:0E05C0007006031DE42AE62AC803BA2A0800C2
:1005CE0083124508C7004608C8004708D7006A21AD
:1005DE0070088312C900CA0100304A06031DF92AA9
:1005EE0000304906031DFC2A202B0330FC009730F7
:1005FE00FD00FD0B002BFC0B002B0000000049083A
:10060E00D700D521C70A0319C80A8030F000803000
:10061E0048067002031D152B4708FF3C0318182BC4
:10062E00202B00304A06031D1E2B00304906031DE9
:04063E00EC2A08009A
:1006420083124508D70055217008C700C601460825
:10065200450784000008D700D521C60A8030460627
:0E066200F000803047067002031C282B0800B1
:100670000A308312D700D5210D30D700D5210800CC
:1006800080308312F000803046067002031D4A2B32
:100690004508003C03185B2B0330FC009730FD003D
:1006A000FD0B502BFC0B502B000000000130C5024D
:0806B000031CC603402B0800E7
:1006B8004F218A110A128000840AB70A0319B80A5E
:0806C800F003031D5C2B080088
:1006D000F03083129F05F03083169F0483129F171A
:1006E0004508F000F00D7010F00D701070089F04B8
:1006F0001F1473219F149F1C7F2B00007B2B1F1046
:100700001E08F100F00183161E08F0040030F10409
:020710000800DF
:1007120083124508C3004608F0000130F200700859
:100722000319972BF20D7210FF3E912B7208B9003C
:100732007209B5004708F1000130F0007108031991
:10074200A62BF00D7010FF3EA02B7008BF00F00921
:100752007008C00080304507840072088004700869
:100762008005B6014C080319B72BB6098413360865
:10077200003A0319BF2B40088005C12B3F088004B3
:10078200CD21E830F4000330F500F601F70196219F
:100792007008CD007108CE007208CF007308D00037
:1007A2004808F0004908F1004A08F2004B08F3003B
:1007B200F00DF10DF20DF30D7010F00DF10DF20DC3
:1007C200F30D70100A30F400F501F601F7019621DD
:1007D2007008D1007108D2007208D3007308D400E7
:1007E2007008F4007108F5007208F6007308F7004B
:1007F2004D08F0004E08F1004F08F2005008F300D7
:100802000E227008D5007108D6007108F400F501B7
:10081200740875040319102C0230F0000800550802
:10082200B3005108F4005208F5005308F6005408CA
:10083200F7004D08F0004E08F1004F08F200500892
:10084200F3000E227808F0007908F1007A08F2002D
:100852007B08F3007008CD007108CE007208CF004B
:100862007308D0005108F5005208F6005308F7004B
:100872005408F800F80CF70CF60CF50CF813781B7A
:10088200F81780307806F400803073067402031D76
:10089200542C72087702031D542C71087602031D32
:1008A200542C700875020318572CB30A3308F10050
:1008B200F10CF1137108B400073071020318642CB3
:0A08C2000130F0000800F00108000A
:1008CC00753083168F001D30850020309500960101
:1008DC005C309F0083129F019F171F131F161F145C
:0808EC00FF3099008B010800A8
:1008F40021308312A0003030A1003130A200323008
:10090400A3003330A4003430A5003530A6003630BF
:10091400A7003730A8003830A9003930AA00303099
:10092400AB003130AC003230AD003330AE00343087
:10093400AF003530B0003630B100B2016624851600
:100944000530C500003005180130C6000030851898
:100954000130C7008030C8002530C900CA01CB016E
:10096400CC0189237008BC007008003C0318D92C02
:10097400BD01BE01203085060230FB000430FC00BE
:10098400BA30FD00FD0BC42CFC0BC42CFB0BC42C97
:100994000000BD0A0319BE0A80303E06F000803014
:1009A4007002031DD72C14303D02031CBC2CC5015E
:1009B400C601E72238233030C5000030C600E722E4
:1009C4000230C500682370088312BA007108BB00A6
:1009D4007008C5007108C6002008C700A8222008B6
:1009E400C50021230930D700D5214030C50000308F
:1009F400C600E7220330C500682370088312C100D3
:100A04007108C2007008C5007108C6002008C7003C
:100A1400A8222008C50021230930D700D521851D2F
:100A2400222D0330FB008A30FC005530FD00FD0B05
:100A3400192DFC0B192DFB0B192D00000000272D7F
:100A44003A08C5003B08C6004023382320308506F9
:040A5400DD2C2B2D3D
:02400E00C400EC
:104200002000560065007200730069006F006E00A8
:1042100020003000390020006A0061006E00760046
:1042200020003200300031003100200050006100D9
:1042300075006C0046006A0075006A006F0020007F
:104240003100320046003600380033005F00320093
:1042500065006D002E004300200020000000FF00DC
:1042600056004F004C005400200041004E00320028
:1042700020004700500031003D000000FF00FF001B
:1042800056004F004C005400200041004E00330007
:1042900020004700500034003D000000FF00FF00F8
:1042A000FF00FF00FF00FF00FF00FF00FF00FF0016
:1042B000FF00FF00FF00FF00FF00FF00FF00FF0006
:1042C000FF00FF00FF00FF00FF00FF00FF00FF00F6
:1042D000FF00FF00FF00FF00FF00FF00FF00FF00E6
:1042E000FF00FF00FF00FF00FF00FF00FF00FF00D6
:1042F000FF00FF00FF00FF00FF00FF00FF00FF00C6
:104300007000610075006C0066006A0075006A004C
:104310006F000000FF00FF00FF00FF00FF00FF0034
:1043200052005300320033003200200039003600C2
:10433000300030000000FF00FF00FF00FF00FF0022
:104340007200FF00FF00FF00FF00FF00FF00FF0002
:10435000FF00FF00FF00FF00FF00FF00FF00FF0065
:10436000FF00FF00FF00FF00FF00FF00FF00FF0055
:10437000FF00FF00FF00FF00FF00FF00FF00FF0045
:10438000FF00FF00FF00FF00FF00FF00FF00FF0035
:10439000FF00FF00FF00FF00FF00FF00FF00FF0025
:1043A000FF00FF00FF00FF00FF00FF00FF00FF0015
:1043B000FF00FF00FF00FF00FF00FF00FF00FF0005
:1043C000FF00FF00FF00FF00FF00FF00FF00FF00F5
:1043D000FF00FF00FF00FF00FF00FF00FF00FF00E5
:1043E000FF00FF00FF00FF00FF00FF00FF00FF00D5
:1043F000FF00FF00FF00FF00FF00FF00FF000000C4
:00000001FF
